:1000000098C0B1C0B0C05EC796C62FC7D4C600C7DF
:1000100065C611C6A8C065C8A6C02DC8EEC0A3C0DD
:10002000A2C0A1C0A0C0D1C2D5C2EAC258C457C4A0
:10003000FFC3E6C346C457C372C398C3BFC3FDC260
:100040000BC323C339C32F6572726F722F6D736731
:100050006C656E6774682F002F6572726F722F74F3
:10006000797065746167322F002F6572726F722F1D
:1000700074797065746167332F002F6572726F72C7
:100080002F74797065746167342F002F6572726FF9
:10009000722F6D736773697A652F002F6572726FA7
:1000A000722F636865636B73756D002F746573746D
:1000B00068616E646C657200000001000800200039
:1000C0004000800000010004000001000800400022
:1000D000000100043031323334353637383941428B
:1000E00043444546002F70776D002F6F7574002FC5
:1000F000696E32002F696E33002F696E34002F69EC
:100100006E35002F696E36002F696E37002F6164DF
:100110006330002F61646331002F61646332002F0C
:1001200061646333002F61646334002F616463355D
:10013000000011241FBECFE5D4E0DEBFCDBF10E02C
:10014000A0E6B0E0E2EFFBE102C005900D92A03620
:10015000B107D9F711E0A0E6B0E001C01D92A437C5
:10016000B107E1F77BCC4CCF96B1987F982B96B92D
:10017000089527B12F73992736E0880F991F3A9574
:10018000E1F7282B27B90895379A359886E0ECDFF8
:1001900081E0EFDF3D98339A10923501789408950D
:1001A00033983798089597B1907E8F71982B97B9AF
:1001B0000895349A369A089586B19927807490707C
:1001C00008951092350197B1907E8F71982B97B951
:1001D000349A369A3699FECF84B1282F332785B1C9
:1001E0009927982F8827822B932B0895EADF9695DD
:1001F000879596958795992708951F920F920FB628
:100200000F9211248F938FEF809335018F910F9070
:100210000FBE0F901F901895AFD660E072EC81E092
:1002200090E07DD6089599278130910579F082304C
:1002300091051CF4892B21F01CC00297A1F019C074
:10024000BAD66CE2ECD7B7D669E618C0B4D66CE281
:10025000E6D7B1D669E6E3D7AED669E6E0D7ABD646
:1002600060E0DDD70895A7D66CE2D9D7A4D663E7BE
:1002700005C0A1D66CE2D3D79ED66EE4D0D79BD66C
:1002800060E0ECCF0F931F93CF93DF93EC0100E07E
:10029000FE01219614918FD6612FC1D70F5F1123D4
:1002A000B9F7802F992783709070892B51F083D6EE
:1002B00060E0B5D70F5F802F992783709070892BEE
:1002C000B1F7DF91CF911F910F9108951F93CF93B5
:1002D000DF93EC01162F6FD66EEBA1D720E0FE0165
:1002E0008491882329F02F5FFE01E20FF11DF8CFE2
:1002F0002F5F822F992783709070892B11F02C7FAC
:100300002C5F120F58D6612F8AD7DF91CF911F91A2
:1003100008950F931F93CF93DF93EC0100E01991A1
:100320004AD6612F7CD70F5F1123C9F7802F9927F9
:1003300083709070892B51F03ED660E070D70F5FCC
:10034000802F992783709070892BB1F7DF91CF911F
:100350001F910F9108950F931F93CF93DF9300E0A8
:1003600012E005C028D6BE0149D7080F1F5FC12F74
:10037000DD2721D6FC0184819581C817D90790F328
:100380001AD6602F4CD7DF91CF911F910F9108950E
:100390000F931F93CF93DF938C01EB0160E0FE017D
:1003A0008491882329F06F5FFE01E60FF11DF8CFDD
:1003B0006F5F862F992783709070892B11F06C7F67
:1003C0006C5F6C5FC80182DFC8015CDF82E02BDFFD
:1003D000CE0158DFC0DF47D6809157018823E1F373
:1003E000DF91CF911F910F9108950F931F93CF939A
:1003F000DF938C01EB0160E08881882331F06F5F2F
:10040000FE01E60FF11D8081F8CF6F5F862F9927DF
:1004100083709070892B11F06C7F6C5F6C5FC801EA
:1004200055DFC8012FDF82E0FEDECE0172DF93DFF1
:100430001AD6809157018823E1F3DF91CF911F9164
:100440000F910895EF92FF920F931F93CF93DF9335
:10045000CDB7DEB728970FB6F894DEBF0FBECDBF7D
:100460007C0149835A836B837C830D831E832F8396
:1004700038876CE02BDFC70105DF81E0D4DE9BD538
:100480006C81CDD698D56B81CAD695D5FE013196B3
:100490006181C5D690D56981C2D68DD56885BFD614
:1004A0008AD56F81BCD687D56E81B9D684D56D814A
:1004B000B6D651DFD8D5809157018823E1F328962D
:1004C0000FB6F894DEBF0FBECDBFDF91CF911F9165
:1004D0000F91FF90EF9008950F931F93CF93DF93A9
:1004E000CDB7DEB724970FB6F894DEBF0FBECDBFF1
:1004F0008C0149835A836B837C8368E0E7DEC80103
:10050000C1DE80E090DE57D56C8189D654D56B81F1
:1005100086D651D5FE013196618181D64CD569814F
:100520007ED619DFA0D5809157018823E1F3249668
:100530000FB6F894DEBF0FBECDBFDF91CF911F91F4
:100540000F9108950F931F938C0160E0BFDEC801E7
:1005500099DE01DF88D5809157018823E1F31F914F
:100560000F91089510926000109244011092420180
:1005700010924A01109249011092A2001092A1001B
:100580001092430140E450E061E670E086E391E0C0
:10059000E6D5E1E6F0E08FE31192815087FFFCCFD2
:1005A00008959093A2008093A10008950F931F9344
:1005B000282F809160009927AA27BB27FC0140972C
:1005C00008F08DC1ED5EFF4F09942E3B09F089C103
:1005D00081E02BC120934401109242012F3310F48B
:1005E00082E023C1822F9927AA27BB278C019D0176
:1005F0004FE350E060E070E086E490E023DF43C02A
:1006000080914201222349F0E82FFF27EF59FF4F45
:1006100020838F5F8093420164C1E82FFF27EF5949
:10062000FF4F20838F5F80934201992783709070E2
:10063000892B09F056C18CE0F8C080914201E82F67
:10064000FF27EF59FF4F20838F5F809342012C32A9
:1006500009F053C08DE0E9C080914201E82FFF27E7
:10066000EF59FF4F20838F5F80934201293611F4A9
:100670008EE0DBC0822F9927AA27BB27AC01BD01E2
:1006800088E590E029DF87E0D0C080914201E82F23
:10069000FF27EF59FF4F20838F5F80934201222372
:1006A00011F48FE0C2C0822F9927AA27BB27AC0183
:1006B000BD0189E690E0E6CF80914201E82FFF2757
:1006C000EF59FF4F20838F5F80934201222311F463
:1006D00088E0ABC0822F9927AA27BB27AC01BD01B8
:1006E0008AE790E0CFCF80914201E82FFF27EF59B2
:1006F000FF4F20838F5F80934201822F9927AA2783
:10070000BB27B82FAA279927882780934501909364
:100710004601A0934701B093480189E086C08091CB
:100720004201E82FFF27EF59FF4F20838F5F80930F
:100730004201822F9927AA27BB27AC013327222702
:100740008091450190914601A0914701B0914801E7
:10075000822B932BA42BB52B8093450190934601BC
:10076000A0934701B09348018AE05FC080914201A5
:10077000E82FFF27EF59FF4F20838F5F80934201BF
:10078000822F9927AA27BB272227382F492F5A2F94
:100790008091450190914601A0914701B091480197
:1007A000822B932BA42BB52B80934501909346016C
:1007B000A0934701B09348018BE037C0809142017C
:1007C000E82FFF27EF59FF4F20838F5F809342016F
:1007D0003327442755278091450190914601A091E8
:1007E0004701B0914801822B932BA42BB52B80930A
:1007F000450190934601A0934701B093480114C06E
:1008000080914201E82FFF27EF59FF4F2083E82F07
:10081000EF5FE093420180914401E81709F061C065
:10082000FF27EF59FF4F108285E08093600059C089
:100830008091420140914401841759F09927AA27D9
:10084000BB275527662777278C019D018BE890E011
:1008500036C01092430190E0941750F4392FE1E62E
:10086000F0E0942F8191380F9150E1F730934301DC
:10087000809143018217C1F48091A1009091A20060
:10088000892B69F18091450190914601A091470122
:10089000B0914801E091A100F091A200AC01BD012E
:1008A00081E690E009951BC09927AA27BB27422F14
:1008B0005527662777278C019D018BE990E0C2DDE3
:1008C0000EC0809142018F5F80934201282F332711
:1008D00080914401992701962817390711F4109245
:1008E00060001F910F9108951F93182F9927AA2731
:1008F000BB27AC01BD018BEA90E0EEDD812F56DE17
:100900001F910895039665E070E00FD9CB01AA27E7
:10091000BB2724E0880F991FAA1FBB1F2A95D1F778
:10092000009711F00197FCCF0895873040F4E82F2D
:10093000FF27EE0FFF1FED55FF4F10821182089524
:10094000089593B7987F982B93BF089510924B0109
:1009500010924C0110924D0110924E01089582E0C8
:10096000F0DF12BE89B7816089BFF0DF08959EB5C0
:10097000987F982B9EBD089583E0F9DF1DBC1CBCB9
:1009800089B7846089BF089595B5987F982B95BDE8
:100990000895109253011092540110925501109233
:1009A0005601089584E0F0DF14BC89B7806489BFE4
:1009B000F0DF0895CF93C0E08C2FB7DFCF5FC73053
:1009C000D8F3CDDFD9DFEEDF7894CF91089583B7E8
:1009D000E82FFF27E770F070EE0FFF1FE853FF4F7F
:1009E0008591949108958EB5E82FFF27E770F070F8
:1009F000EE0FFF1FE853FF4F85919491089585B541
:100A0000E82FFF27E770F070EE0FFF1FE854FF4F4D
:100A1000859194910895873040F4E82FFF27EE0FD9
:100A2000FF1FED55FF4F6083718308950895DF9296
:100A3000EF92FF920F931F93CF93DF93EC01D2B607
:100A400010924F01109250011092510110925201D8
:100A5000BEDF9C014427552760E074E284EF90E0FC
:100A6000ADD8293B8DE8380786E0480780E0580775
:100A7000B0F487E2C131D80790F4CE01AA27BB2792
:100A8000BC01CD0133D8DC01CB01BC01CD0128EE86
:100A900033E040E050E070D8FA01E9010FC07E0178
:100AA00000271127CA01B90128EE33E040E050E0E9
:100AB00063D8C801B7011AD8FC01EB0180914F013E
:100AC00090915001A0915101B09152012227382FED
:100AD000492F5A2F82B79927AA27BB27282B392BB2
:100AE0004A2B5B2BCD0DD11DE11DF11D2C173D07B0
:100AF0004E075F0758F580914F0190915001A091EA
:100B00005101B091520185B78F7885BF85B7806854
:100B100085BF889585B78F7785BF80914F0190916C
:100B20005001A0915101B0915201BA2FA92F982FD5
:100B3000882722B7332744275527822B932BA42BB2
:100B4000B52B8C179D07AE07BF07A8F2DF91CF9199
:100B50001F910F91FF90EF90DF90089580914B01CE
:100B600090914C01A0914D01B0914E01BC01CD017D
:100B700008958091530190915401A0915501B09135
:100B80005601BC01CD010895893031F48FB58260E2
:100B90008FBD8FB58E7F0AC08A3019F48FB5826001
:100BA00002C08FB58D7F8FBD8FB581608FBD1BBC9F
:100BB0001ABC19BC18BC08959C018FB58E7F8FBDDF
:100BC0008FB582608FBD8EB588608EBD8EB5806119
:100BD0008EBD37BD26BD1BBC1ABC19BC18BC089500
:100BE0008FB58F778FBD8FB58F7B8FBD08958FB5F4
:100BF0008F7D8FBD8FB58F7E8FBD08958FB58D7F13
:100C00008FBD8FB58E7F8FBDEBDFF1DF08958FB580
:100C100080688FBD8FB58F7B8FBD08958FB5806243
:100C20008FBD8FB58F7E8FBD08959BBD8ABD089502
:100C300099BD88BD08951F920F920FB60F9211248F
:100C40002F933F934F935F936F937F938F939F93D4
:100C5000AF93BF93EF93FF9380914B0190914C0121
:100C6000A0914D01B0914E010196A11DB11D80933F
:100C70004B0190934C01A0934D01B0934E01809194
:100C80004F0190915001A0915101B09152010196F4
:100C9000A11DB11D80934F0190935001A09351016C
:100CA000B09352018091A3009091A400892B29F068
:100CB000E091A300F091A4000995FF91EF91BF91FD
:100CC000AF919F918F917F916F915F914F913F91E4
:100CD0002F910F900FBE0F901F9018951F920F929B
:100CE0000FB60F9211242F933F934F935F936F93FF
:100CF0007F938F939F93AF93BF93EF93FF938091D5
:100D0000A5009091A600892B29F0E091A500F09113
:100D1000A6000995FF91EF91BF91AF919F918F919F
:100D20007F916F915F914F913F912F910F900FBEE7
:100D30000F901F9018951F920F920FB60F921124CB
:100D40002F933F934F935F936F937F938F939F93D3
:100D5000AF93BF93EF93FF93809153019091540110
:100D6000A0915501B09156010196A11DB11D80932E
:100D7000530190935401A0935501B0935601809173
:100D8000AD009091AE00892B29F0E091AD00F0917B
:100D9000AE000995FF91EF91BF91AF919F918F9117
:100DA0007F916F915F914F913F912F910F900FBE67
:100DB0000F901F9018951F920F920FB60F9211244B
:100DC0002F933F934F935F936F937F938F939F9353
:100DD000AF93BF93EF93FF938091A7009091A800EA
:100DE000892B29F0E091A700F091A8000995FF91C7
:100DF000EF91BF91AF919F918F917F916F915F9193
:100E00004F913F912F910F900FBE0F901F9018950B
:100E10001F920F920FB60F9211242F933F934F936F
:100E20005F936F937F938F939F93AF93BF93EF9352
:100E3000FF938091A9009091AA00892B29F0E0915D
:100E4000A900F091AA000995FF91EF91BF91AF9190
:100E50009F918F917F916F915F914F913F912F91D2
:100E60000F900FBE0F901F9018951F920F920FB604
:100E70000F9211242F933F934F935F936F937F9320
:100E80008F939F93AF93BF93EF93FF938091AB00AA
:100E90009091AC00892B29F0E091AB00F091AC006F
:100EA0000995FF91EF91BF91AF919F918F917F91A4
:100EB0006F915F914F913F912F910F900FBE0F90C7
:100EC0001F9018951F920F920FB60F9211242F9317
:100ED0003F934F935F936F937F938F939F93AF93C2
:100EE000BF93EF93FF938091AF009091B000892B57
:100EF00029F0E091AF00F091B0000995FF91EF91DA
:100F0000BF91AF919F918F917F916F915F914F9121
:100F10003F912F910F900FBE0F901F901895DC01FD
:100F2000CB0173E0880F991FAA1FBB1F7A95D1F7D9
:100F30009C01AD01220F331F441F551F80509C4D53
:100F4000AB40BF4FBC01CD0117D6DA01C9010197F3
:100F500089B9892F992780BD089540E450E061EB5D
:100F600070E088E591E0FBD040E450E061EF70E094
:100F700081E691E0F4D00895F0DF109232011092F2
:100F8000310188ED8AB960E875E280E090E0C7DF62
:100F90008FEF809357011092600110926A011092B6
:100FA00069017894089590933201809331010895F6
:100FB00088E591E0089581E691E00895982F809169
:100FC00057018823E1F39CB9109257010895CF93FC
:100FD000DF93EC0180915A0190915B01009761F0E1
:100FE00080915C0190915D01009731F088E591E07E
:100FF000C0D088838FEF90E0DF91CF910895CF9399
:10100000DF93CDB7DEB721970FB6F894DEBF0FBEE2
:10101000CDBFCE010196DBDF882319F089819927A6
:1010200002C08FEF9FEF21960FB6F894DEBF0FBE80
:10103000CDBFDF91CF91089510925D0110925C01B8
:10104000089580915C0190915D01892B19F48FEFD7
:1010500090E0089580E090E008950895682F81E67B
:1010600091E0DDD008958FEF8093600181E691E0FB
:1010700080D0A4DF08951F920F920FB60F92112413
:101080002F933F934F935F936F937F938F939F9390
:10109000AF93BF93EF93FF9380916001882369F032
:1010A0008091650190916601892B29F081E691E09C
:1010B00060D08CB905C0109260018FEF809357010A
:1010C000FF91EF91BF91AF919F918F917F916F9120
:1010D0005F914F913F912F910F900FBE0F901F90F6
:1010E00018951F920F920FB60F9211242F933F93D2
:1010F0004F935F936F937F938F939F93AF93BF9320
:10110000EF93FF936CB18091310190913201892B63
:1011100039F0E0913101F0913201862F09950EC02E
:1011200088E591E07CD0882349F480916901909111
:101130006A01019690936A0180936901FF91EF9192
:10114000BF91AF919F918F917F916F915F914F91DF
:101150003F912F910F900FBE0F901F901895FC019B
:1011600060837183428353831682178214821582AF
:101170000895CF93DF93EC01E0E02C813D812115B0
:101180003105B1F08E819F81E881F981E80FF91F67
:10119000E08101968E839F836A817B818617970702
:1011A00018F0C3D48E839F83215030402C833D831D
:1011B0008E2F9927DF91CF910895CF93DF93FC0174
:1011C000EB01248135816217730798F4868197813A
:1011D000860F971F8683978362817381861797078F
:1011E00018F0A3D4868397832C1B3D0B248335836F
:1011F00002C014821582DF91CF910895FC0186818F
:10120000978122813381860F971FB9018ED4019077
:10121000F081E02DE80FF91F808199270895CF9381
:10122000DF93EC01462F2C813D816A817B8126175B
:10123000370790F48E819F81820F931F76D4E881C7
:10124000F981E80FF91F40838C819D8101968C8381
:101250009D838FEF90E002C080E090E0DF91CF911E
:101260000895FC0140E050E0248135818281938122
:101270002817390710F441E050E0CA010895FC0135
:101280001482158208959093340180933301089558
:10129000E0913301F091340109950895CF93DF93E4
:1012A000EC01892B61F08881882349F0E0913301BA
:1012B000F09134018991099588818823B9F7DF91EC
:1012C000CF910895EF92FF920F931F93CF93DF93E7
:1012D000EC017A0120E030E0892B01F1C9012F5F98
:1012E0003F4F8617970718F489918823B9F720E0B4
:1012F00030E02E153F0590F4888189010F5F1F4F64
:10130000E0913301F0913401882311F0219601C05E
:1013100080E2099598010E151F0570F3DF91CF91BA
:101320001F910F91FF90EF900895CF93DF93EC0101
:10133000009779F0FC0121968491882351F0E09187
:101340003301F09134010995FE012196849188239F
:10135000B1F7DF91CF910895E0913301F09134011D
:101360008DE00995E0913301F09134018AE009950F
:101370000895E82FFF27EF70F070EC52FF4F849133
:10138000E0913301F0913401099508951F93182FCE
:1013900082958F70EEDF812FECDF1F9108950F9300
:1013A0001F938C01812F9927F1DF802FEFDF1F9191
:1013B0000F910895EF92FF920F931F937B018C0181
:1013C000C801AA27BB27EBDFC701E9DF1F910F91F7
:1013D000FF90EF9008952F923F924F925F926F92FD
:1013E0007F928F929F92AF92BF92CF92DF92EF92B5
:1013F000FF920F931F93CF93DF93CDB7DEB7A297E2
:101400000FB6F894DEBF0FBECDBF69A3C42E2AA3CA
:1014100027013801442351F017FF08C0EE24FF24B0
:101420008701E418F5080609170902C08301720153
:1014300099A1692F772767FD709561507040CC2086
:1014400011F061507040D62E18A22FE1222E312CBF
:101450002C0E3D1E882E992487FC9094A92CB92C23
:10146000C801B701A501940187D3DC01CB01FC01C0
:10147000EC52FF4F84918F8FC801B701A5019401F1
:101480007BD379018A01DA94AFEFDA1629F1DA9485
:10149000C1010197E114F10401051105B1F01C012E
:1014A000C801B701A501940167D3DC01CB01FC01A0
:1014B000EC52FF4F8491F1018083C801B701A5016F
:1014C00094015AD379018A0104C01C01EAA1DC010C
:1014D000EC93FFEFDF16D9F6CC20B9F077FE05C00C
:1014E0008DE2D1018E931D0110C0C101019714142A
:1014F0001504160417042CF41C018BE2F1018083FF
:1015000004C01C0180E2D1018C93D9A0DA94BFEF12
:10151000DB1661F0E0913301F0913401D1018D913E
:101520001D010995DA94BFEFDB16A1F7A2960FB65D
:10153000F894DEBF0FBECDBFDF91CF911F910F9109
:10154000FF90EF90DF90CF90BF90AF909F908F90E3
:101550007F906F905F904F903F902F9008957F9273
:101560008F929F92AF92BF92CF92DF92EF92FF92B3
:101570000F931F93CF93DF93CDB7DEB77888C988D9
:10158000DA8863E1A62EB12CAC0EBD1E08C08823FC
:1015900009F47DC0E0913301F09134010995960181
:1015A0002F5F3F4F772021F0F6016901849103C03E
:1015B000F60180816901853251F72F5F3F4F772017
:1015C00021F0F6016901849103C0F601808169016F
:1015D000282F332727FD30952436310591F0253605
:1015E000310524F42336310529F0D4CF28373105CD
:1015F00081F0D0CFF50122E030E0A20EB31E808151
:10160000C9CF5AE0852E912C40E1E42E47E2F42E1A
:1016100004C030E1E32EF12C4701F50122E030E077
:10162000A20EB31E008111818436D1F417FF09C0C8
:10163000109501951F4FE0913301F09134018DE237
:10164000099532E0E316F10458F00E151F0540F439
:10165000C7016AE070E069D27B0162307105A8F7CA
:10166000C801B70162D2FB01EC52FF4F8491E091B7
:101670003301F09134010995C801B70156D28C01AC
:10168000C701B40152D27B01672B51F788CF80E0AC
:1016900090E0DF91CF911F910F91FF90EF90DF903D
:1016A000CF90BF90AF909F908F907F900895282FFC
:1016B000332760FF0DC081E090E002C0880F991FC2
:1016C0002A95E2F7982F909588B3892388BB0895CF
:1016D00081E090E002C0880F991F2A95E2F728B3B5
:1016E000282B28BB08950895EF92FF920F931F9324
:1016F000CF93DF93EC017A018B0144E050E065EE7B
:1017000070E0E6D1892BA9F4FE0101900020E9F7F1
:101710003697EC17FD0709F06FC08C81803319F400
:101720008E2D992741C0813309F066C08E2D9927EF
:101730005BC044E050E06AEE70E0CE01C9D1AC017C
:10174000892B09F059C0FE0101900020E9F731977B
:10175000EC1BFD0BE530F10519F0369709F04CC094
:101760008C81282F332727FD30952833310559F0F8
:101770002933310524F421333105C1F03DC029332B
:10178000310521F039C06E2D80E035C081E090E058
:10179000A0E0B0E0E822F9220A231B23EF2811F091
:1017A000CA0102C08FEF90E040DA26C08D819927F0
:1017B00087FD909581339105C9F0823391051CF422
:1017C000C09721F019C0C297A1F016C081E090E047
:1017D000A0E0B0E0E822F9220A231B23EF2811F051
:1017E000CA0102C08FEF90E023DA06C06E2D83E0BD
:1017F00002C06E2D84E05BDFDF91CF911F910F91CE
:10180000FF90EF9008951F93CF93DF9310B3C12FF4
:10181000DD279E01247030708091730199278470B8
:10182000907028173907A1F0CE0196958795969567
:10183000879521E030E082279327AA27BB27817074
:101840009070A070B070AC01BD018FEE90E044D6F6
:101850009E01287030708091730199278870907074
:1018600028173907A9F0CE0163E0969587956A9508
:10187000E1F721E030E082279327AA27BB27817078
:101880009070A070B070AC01BD0184EF90E024D6E0
:101890009E01207130708091730199278071907042
:1018A00028173907A9F0CE0154E0969587955A95E7
:1018B000E1F721E030E082279327AA27BB27817038
:1018C0009070A070B070AC01BD0189EF90E004D6BB
:1018D0009E01207230708091730199278072907000
:1018E00028173907A9F0CE0145E0969587954A95C6
:1018F000E1F721E030E082279327AA27BB278170F8
:101900009070A070B070AC01BD018EEF90E0E4D596
:101910009E012074307080917301992780749070BB
:1019200028173907A9F0CE0136E0969587953A95A4
:10193000E1F721E030E082279327AA27BB278170B7
:101940009070A070B070AC01BD0183E091E0C4D58F
:10195000C078D07080917301992780789070C817F3
:10196000D907A9F0812F992787FD9095A92FB92F25
:1019700080959095A095B0958827B7FD8395992778
:10198000AA27BB27AC01BD0188E091E0A5D5109343
:101990007301DF91CF911F9108951F93182F26D4C3
:1019A000382F9927412F5527FA01E559FE4F2081FD
:1019B000821B91090896419708F44EC0308342304B
:1019C000510531F1433051053CF44115510571F099
:1019D00041305105A1F040C04430510559F1443027
:1019E0005105FCF04530510571F136C0832F992720
:1019F000AA27BB27AC01BD018DE091E02CC0832F4D
:101A00009927AA27BB27AC01BD0183E191E023C040
:101A1000832F9927AA27BB27AC01BD0189E191E05B
:101A20001AC0832F9927AA27BB27AC01BD018FE1DC
:101A300091E011C0832F9927AA27BB27AC01BD01D4
:101A400085E291E008C0832F9927AA27BB27AC0124
:101A5000BD018BE291E040D51F910895CEE5D4E021
:101A6000DEBFCDBFA7D711BA8FEF82BBB89AC0989F
:101A7000BB9AC398BC9AC49887D3B99ABA9A7CD7B0
:101A800088E082D8C4D8CAD880E090E0CED880E080
:101A900090E0CED871DA60E072EC81E090E03FDA5D
:101AA000BBD360D584E79BE07CD510E0ACDE812F12
:101AB00074DF812F9927019666E070E04AD0182FD5
:101AC000CE01019684DA882389F389816FD5EECF20
:101AD000FB01DC014150504030F08D9105908019A0
:101AE00019F40020B9F7881B990B0895629FD00163
:101AF000739FF001829FE00DF11D649FE00DF11DC9
:101B0000929FF00D839FF00D749FF00D659FF00D77
:101B10009927729FB00DE11DF91F639FB00DE11D64
:101B2000F91FBD01CF0111240895AA1BBB1B51E170
:101B300007C0AA1FBB1FA617B70710F0A61BB70B3D
:101B4000881F991F5A95A9F780959095BC01CD01E2
:101B5000089597FB092E07260AD077FD04D0E5DF0C
:101B600006D000201AF4709561957F4F0895F6F71E
:101B7000909581959F4F0895A1E21A2EAA1BBB1B39
:101B8000FD010DC0AA1FBB1FEE1FFF1FA217B30749
:101B9000E407F50720F0A21BB30BE40BF50B661F5F
:101BA000771F881F991F1A9469F760957095809523
:101BB00090959B01AC01BD01CF01089597FB092EC3
:101BC00005260ED057FD04D0D7DF0AD0001C38F40C
:101BD00050954095309521953F4F4F4F5F4F089559
:101BE000F6F790958095709561957F4F8F4F9F4F39
:021BF000089556
:00000001FF
